:020000020000FC
:1000000003C002C001C0ABC0C0E00C2ECCEFC7BB28
:10001000C0E0C8BBCBE0C8B9CFE7C1BB80E0C1E05E
:10002000C3BFF894909A9598CFEFC7BBC0E0C8BB08
:10003000969A90E0A9E111278EE688BB0DE0015069
:10004000F1F700008DE688BB0DE00150F1F715597E
:1000500000F49150A04080F7939A9698CCEFC7BBDC
:10006000C0E0C8BB8CE688BB90E0AAE09150A040FD
:10007000E8F7CAE03C2E4C2E5C2E6C2E02BE1124FA
:10008000BB279298DD27789490E0A4E6B23021F067
:100090009150A040D8F739C0CFE07C2E48D0A8F1CD
:1000A000DE3729F0DE3F19F07A94C1F72EC02227FF
:1000B0003327E8E0C8E07C2E3AD038F146D07A9475
:1000C000D9F7CD2FC083E395E231A1F7C8E07C2EAC
:1000D0002ED0D8F07A94E1F7CD2FCE3711F0CE3F65
:1000E000A1F4F894959AADE07DD0AAE07BD0E8E049
:1000F00060816DD06FD0A0E275D0E395E431C1F797
:10010000C22FC32B09F4909808C0F8949598ADE0DD
:1001100069D0AAE067D0AFE365D0F89490E0A4E19D
:1001200084E68150F0F79150A040D0F77ACF99271C
:10013000C22DCC2321F49A95D9F708940895C17063
:100140002224C795D79588940895CD2FCC1F221FC0
:10015000331F20F4C0E13C27C1E22C2708957FB76C
:1001600062B702BE919A6555652C542C432C362EED
:10017000640D650D660D643130F4623208F005C01F
:100180009598E89402C0959A6894661F661F6E7FE2
:1001900068BBB03031F41394612D6431A9F4B1E03F
:1001A00013C0B13029F486F4B2E06FEF162E0CC004
:1001B00013949298612D6F70673031F416F062E0FD
:1001C00001C063E0262E929A91987FBF1895A62FC2
:1001D000A29502C0A62F00C0AF70AA5FA4FDA95FC0
:1001E000A65D00C0BBE0BB3021F0B33020F0A79586
:1001F00010F0949A01C0949899EF9A95000000002D
:08020000E1F7BA9581F70895BA
:00000001FF
